:100000000C942A000C9447000C9447000C94470071
:100010000C9447000C9447000C9447000C94470044
:100020000C9447000C947F000C9447000C94D00172
:100030000C94FA010C9447000C9447000C94470070
:100040000C9447000C9447000C9447000C94470014
:100050000C94470011241FBECFE5D4E0DEBFCDBF16
:1000600010E0A0E6B0E0ECEDF5E002C005900D92E6
:10007000A037B107D9F710E0A0E7B0E001C01D92AA
:10008000A13DB107E1F70E9454000C94ED020C94DD
:100090000000089581E089BF13BE84E682BF8CE929
:1000A0008CBF85E083BF0895CF93DF9385B38360D2
:1000B00085BB87E690E00E941F020E944A00789468
:1000C0008CE30E94B1008CE10E94AE000E945A01B4
:1000D00080E690E00E945D02CAE6D0E00E94A500A2
:1000E0000E948C02CE010E945D0220E137E280E98D
:1000F00091E00197F1F721503040C9F7EFCF1F92FF
:100100000F920FB60F9211242F933F934F935F934B
:100110006F937F938F939F93AF93BF93EF93FF93CF
:1001200084E682BF0E940E01FF91EF91BF91AF91D3
:100130009F918F917F916F915F914F913F912F91FF
:100140000F900FBE0F901F901895809171009091A5
:10015000720008958091730090E0089580936D007F
:10016000089580936E00089580EE0E9464018823B4
:1001700029F40E94AA0181E090E008950E94AA015A
:1001800080E090E008950F931F930E94B4008823AD
:1001900021F180EE0E94640181E00E94B00181EEB5
:1001A0000E94A6010E94C001809373000E94C001BA
:1001B00090E0982F882790937200809371000091AF
:1001C0007100109172000E94C801080F111D109358
:1001D0007200009371000E94AA011F910F9108956F
:1001E0000E94B4008823C9F080EE0E94640181E07F
:1001F0000E94B00180916D000E94B00180916E005C
:100200000E94B00180EE0E94A60180E00E94B00131
:1002100081E50E94B0010E94AA01089580917400B6
:100220008230C9F0833028F4882351F08130B1F551
:100230000EC08430E9F08430A0F0853079F524C018
:1002400080917000882319F081E0809374000E94EF
:10025000F00082E01EC00E94B4008823F9F083E021
:1002600018C00E94C30084E08093740085E007C03A
:1002700080917500882331F08091750081508093C2
:100280007500089585E005C080917000882321F0F5
:1002900081E080937400089510927400089588237B
:1002A00031F081E0809370000E9460010895109207
:1002B000700008950E94600181E0809370000895AD
:1002C00011B888E480B90895982F84EA86BF06B6ED
:1002D00007FEFDCF81B1887F883029F0803119F089
:1002E00081E090E0089593B984E886BF06B607FEE2
:1002F000FDCF21B1287F283119F480E090E00895E6
:1003000080E090E0203411F081E090E00895982F93
:1003100084EA86BF06B607FEFDCF81B1887F8830AC
:1003200011F08031A9F793B984E886BF06B607FEBD
:10033000FDCF81B1887F803211F0883531F484E9B6
:1003400086BF06B604FEE4CFFCCF08950E94640188
:1003500090E0089584E986BF06B604FCFDCF0895B9
:1003600083B984E886BF06B607FEFDCF81B120E0E1
:1003700030E0887F883211F021E030E0C901089533
:1003800084EC86BF06B607FEFDCF83B190E00895EA
:1003900084E886BF06B607FEFDCF83B190E00895DE
:1003A0001F920F920FB60F9211242F938F939F934A
:1003B000EF93FF939BB12CB1E091B800EF5FEF7129
:1003C0008091B900E81711F482E008C0892F887184
:1003D000E093B800F0E0EA56FF4F20838093BA0024
:1003E000FF91EF919F918F912F910F900FBE0F90E2
:1003F0001F9018951F920F920FB60F9211248F9392
:100400009F93EF93FF939091B6008091B700981758
:1004100061F0E091B700EF5FEF71E093B700F0E0BB
:10042000EA58FF4F80818CB901C05598FF91EF9138
:100430009F918F910F900FBE0F901F901895109263
:10044000B6001092B7001092B8001092B900292F90
:10045000332720BD89B988E98AB986E880BD089527
:100460009091B8008091B900981719F480E091E05C
:100470000895E091B900EF5FEF71E093B900F0E00B
:10048000EA56FF4F20818091BA0090E0982F88278C
:10049000820F911D0895282F9091B6009F5F9F7144
:1004A0008091B7009817E1F3E92FF0E0EA58FF4F89
:1004B00020839093B600559A0895CF93DF93EC0173
:1004C00003C021960E944B0288818823D1F7DF91D7
:1004D000CF910895CF93DF93EC0102C00E944B02AD
:1004E000FE01219684918823C9F7DF91CF91089569
:1004F0008F708A3010F0895C01C0805D0E944B02D1
:1005000008951F93182F82958F700E947802812F73
:100510000E9478021F910895CF93DF93CDB7DEB785
:1005200061970FB6F894DEBF0FBECDBF4AE050E032
:10053000BE016F5F7F4F0E94A8020E945D0261961C
:100540000FB6F894DEBF0FBECDBFDF91CF910895F7
:10055000FB019F01E8944230C4F04532B4F44A30C4
:1005600029F497FB1EF4909581959F4F642F772770
:100570000E94D902805D8A330CF0895D8193CB01A2
:100580000097A1F716F45DE251931082C9010C9413
:10059000C902DC01FC01672F71917723E1F73297E3
:1005A00004C07C916D9370836291AE17BF07C8F34E
:1005B0000895AA1BBB1B51E107C0AA1FBB1FA617AA
:1005C000B70710F0A61BB70B881F991F5A95A9F7FC
:0C05D00080959095BC01CD010895FFCFEF
:1005DC00746163682061756368000D0A0007180078
:00000001FF
